:100000000C94FA000C9420010C9420010C94200113
:100010000C9420010C9420010C9420010C942001DC
:100020000C9420010C9420010C9420010C942001CC
:100030000C9420010C9420010C94F6020C942001E5
:100040000C9420010C9420010C9420010C942001AC
:100050000C9420010C9420010C9420010C9420019C
:100060000C94D6020C9420010C9420010C942001D5
:100070000C9420010C9420010C9420010C9420017C
:100080000C9420010C9420010C9420010C9420016C
:100090000C9420010C9420010C9420010C9420015C
:1000A0000C9420010C9420010C9420010C9420014C
:1000B0000C9420010C9420010C9420010C9420013C
:1000C0000C9420010C9420010C9420010C9420012C
:1000D0000C9420010C9420010C9420010C9420011C
:1000E0000C9420010C9420010C9420010C9420010C
:1000F0000C9420010C9420010C9420010C942001FC
:100100000C9420010C9420010C9420010C942001EB
:100110000C9420010C9420010C9420010C942001DB
:100120000C9420010C9420010C9420010C942001CB
:100130000C9420010C9420010C9420010C942001BB
:100140000C9420010C9420010C9420010C942001AB
:100150000C9420010C9420010C9420010C9420019B
:100160000C9420010C9420010C9420010C9420018B
:100170000C9420010C9420010C9420010C9420017B
:100180000C9420010C9420010C9420010C9420016B
:100190000C9420010C9420010C9420010C9420015B
:1001A0000C9420010C9420010C9420010C9420014B
:1001B0000C9420010C9420010C9420010C9420013B
:1001C0000C9420010C9420010C9420010C9420012B
:1001D0000C9420010C9420010C9420010C9420011B
:1001E0000C9420010C9420010C9420010C9420010B
:1001F0000C94200111241FBECFEFDFE3DEBFCDBF83
:1002000000E00CBF18BE19BE1ABE1BBE10E2A0E073
:10021000B0E2ECE5FCE000E00BBF02C007900D92FD
:10022000A830B107D9F71BBE10E2A8E0B0E201C0C8
:100230001D92AA34B107E1F70E945E030C942C06CC
:100240000C940000E0E0F8E082EA9BE786A397A325
:100250008081807F8760808386818C7F82608683B7
:10026000E0EAF0E08281826082830895A09102201A
:10027000B09103208C91813009F0B0C012968C911E
:100280001297882329F414961C92149720E044C0F6
:1002900014962C91149730E018968C91189790E052
:1002A00004962817390719F414961C92149714967B
:1002B0002C91149730E018968C91189790E0039643
:1002C0002817390711F020E004C012961C921297EB
:1002D00024E414963C911497E32FF0E018968C9147
:1002E000189790E002968E179F074CF0332339F051
:1002F000EA0FFB1F22893F5F14963C9314971496D4
:100300008C911497882341F418962C911897206BA0
:1003100081E014968C931497E0910820F0910920C5
:100320002383438113962C91139730E017968C9179
:10033000179790E004962817390719F413961C9222
:10034000139713962C91139730E017968C9117976B
:1003500090E0039628173907A9F4443481F480E12A
:10036000E0E8F6E0878381E011968C93119713966D
:100370008C9113978F5F13968C93139703C01396EA
:100380001C92139713962C911397E22FF0E0179677
:100390008C91179790E002968E179F074CF02223BE
:1003A00039F0EA0FFB1F40872F5F13962C931397AA
:1003B00013968C911397882381F4842F807F803B40
:1003C00049F44F7017964C93179781E013968C93CE
:1003D000139703C013961C9213971C920895CF9302
:1003E000DF932091042030910520F901838581302D
:1003F000C9F4C0910220D09103208285888740E013
:1004000008C0FE01EA0FFB1FA20FB31F8C91838B64
:100410004F5FA42FB0E0888590E001968A179B0774
:1004200084F720C02091062030910720F9018385B0
:100430008130E1F4C0910220D09103208285888729
:1004400040E008C0FE01EA0FFB1FA20FB31F8C9112
:10045000838B4F5FA42FB0E0888590E001968A17C8
:100460009B0784F7F901138681E08A83DF91CF919E
:100470000895CF93DF932091022030910320D9017A
:1004800011968C911197813069F519968C91813074
:1004900031F0C0910620D091072040E016C0E091D5
:1004A0000020F0910120D9011B968C91828380E27B
:1004B000E0E8F6E0878316C0FE01EA0FFB1FA20FFB
:1004C000B31F19968C9180834F5FF9015781A42F38
:1004D000B0E0852F90E001968A179B076CF75A874A
:1004E00081E08B87D90111961C92DF91CF910895FD
:1004F000A0910420B09105201C968C911C9781300E
:1005000059F51B968C931B9787E08C93E091002004
:10051000F0910120828111968C93119787E61296B3
:100520008C93129788E613968C93139789E614960A
:100530008C93149780E715968C93159781E7169600
:100540008C93169782E717968C93179786E01A96E6
:100550008C931A971C961C920895CF93DF93209149
:10056000022030910320F90181818130E1F4C091B2
:100570000620D091072040E009C0FE01EA0FFB1FD2
:10058000A20FB31F19968C9180834F5FF901578199
:10059000A42FB0E0852F90E001968A179B076CF797
:1005A0005A8781E08B87DF91CF9108951F920F9238
:1005B0000FB60F9208B60F920BB60F92112418BE09
:1005C0001BBE8F93EF93FF93E0910220F0910320E5
:1005D00081E08083FF91EF918F910F900BBE0F9080
:1005E00008BE0F900FBE0F901F9018951F920F928C
:1005F0000FB60F9208B60F920BB60F92112418BEC9
:100600001BBE8F93EF93FF93E0910420F0910520A0
:1006100081E08487FF91EF918F910F900BBE0F9037
:1006200008BE0F900FBE0F901F9018950F931F9349
:100630008FEF8093A00600E01BE082ED90E0F801D0
:1006400086A397A380E09BE063E00E94AE0580E074
:100650009BE060E10E94C80580E09BE061E00E94B1
:10066000A20589E690E0F80180AF91AF1F910F914C
:1006700008958091500082608093500003C081E013
:100680000E942E058091510081FFF9CF0895EF92CD
:100690000F9388E090E260EC78E040E456E020E0E0
:1006A00004E032E0E32E0E94E403E0EAF0E082811D
:1006B0008360828378940F91EF900895E0910020F9
:1006C000F0910120128291E09093600682E3809382
:1006D0008006E0E6F6E094831092452010924620D2
:1006E000E0910220F091032010820E9447030E94B3
:1006F000390380E197E220E233E0F9013197F1F725
:100700000197D9F70E941603E0E0F8E082EA9BE740
:1007100086A397A380910008807F8760809300085C
:10072000809106088C7F826086838091A20082601F
:10073000E0EAF0E08283E0910220F091032082E081
:10074000158A8F5F31968A30D9F782E0E0E8F6E0CB
:1007500084830E9436010E94EF010E9439020E94A8
:100760007802F7CFAF92CF92EF920F93DC01FB01AB
:100770006D937C93119712964D935C9313971496F7
:100780001C921497CC2011F490E001C090E8222331
:1007900011F480E001C080E200650A29902B892BCA
:1007A0008083ED91FC911197E18215961D921C9228
:1007B00016971296ED91FC91139780EA81830F9121
:1007C000EF90CF90AF900895EF920F93DC01FB0173
:1007D0006D937C93119712964D935C9313972223FC
:1007E00011F480E401C080E6802B8083ED91FC91C0
:1007F0001197E1821296ED91FC91139780E4818329
:100800000F91EF900895EF920F931F93FC010083D7
:100810001183E28263837483458356832783108622
:1008200011861F910F91EF900895CF93DF93DC0114
:100830001596CD91DC9116979885ED91FC911197C5
:10084000808184FD05C081E014968C93149724C0A8
:100850008381ED81FE81E90FF11D80839F5F1596F5
:10086000ED91FC9116978781981758F40380F481D5
:10087000E02DE90FF11D8081ED91FC9111978383AB
:100880000BC082810190F081E02D85831596ED915A
:10089000FC91169781E081871596ED91FC91169752
:1008A0009087DF91CF910895CF93DF93DC01EB0127
:1008B00014969C9114971596ED91FC91169730978C
:1008C00029F415966D937C93169710C08185882323
:1008D00011F482E028C0992349F01296ED91FC9121
:1008E0001397848184FD02C081E01DC01596CD93CD
:1008F000DC931697198614961C9214978A81E881C6
:10090000F98186831596ED91FC91169710861596C0
:10091000ED91FC9116970380F481E02D8081ED919B
:10092000FC91838380E0DF91CF910895FC01A08149
:10093000B18113966C930190F081E02D828187FF45
:10094000FDCF83810895CF93DF93EC01FB01611507
:10095000710511F480E037C06D837E834281A081F0
:10096000B181109711F016964C93678190E01AC0F0
:10097000292F30E00380F481E02DE20FF31F808106
:10098000E881F9818383E881F981828187FFFDCF46
:100990008381ED81FE810580F681E02DE20FF31F5A
:1009A00080839F5FED81FE81961710F30190F081A7
:1009B000E02D309709F04583ED81FE816087ED8160
:1009C000FE8181E08187DF91CF9108950F93DF93BE
:1009D000CF930F92CDB7DEB72FB72983F8941BBE04
:1009E000FC0108ED04BF608389818FBF0F90CF9118
:1009F000DF910F910895662311F490E001C090E219
:100A0000482B942BE0E5F0E0928308956F71682BFA
:100A1000E0E5F0E065830895E0E5F0E02081982FBF
:100A20009095922390839081892308950F93DF936B
:100A3000CF930F92CDB7DEB79FB79983F8941BBEC3
:100A4000682B81E490E0FC0108ED04BF608389819C
:100A50008FBF0F90CF91DF910F9108950F93DF9388
:100A6000CF930F92CDB7DEB7209140009FB7998307
:100A7000F8941BBEA0E4B0E0287F282BFD0108ED10
:100A800004BF208399819FBF9C9189230F90CF91B0
:100A9000DF910F910895E0E4F0E09381917F916000
:100AA000982B93830895282F30915600662311F0D8
:100AB000982F01C090E0822F80958323982BE0E54A
:100AC000F0E09683213031F480916800816080935A
:100AD00068000895223029F480916000816080933D
:100AE000600008950F93DF93CF930F92CDB7DEB7D9
:100AF0008FB78983F8941BBE23E083E590E0FC0167
:100B000008ED04BF208389818FBF0F90CF91DF91C3
:100B10000F9108950F93DF93CF930F92CDB7DEB768
:100B20008FB78983F8941BBE21E082E490E0FC013A
:100B300008ED04BF208389818FBF0F90CF91DF9193
:100B40000F910895FC018081807F862B808308951A
:100B5000FC018081807F862B80830895FC01818148
:100B6000887F862B81830895FC018181887F862B75
:100B700081830895FC01838180718062862B838349
:100B80000895FC01838180718062862B83830895A0
:100B9000FC018181607F862B81830895FC01818126
:100BA0006073862B81830895FC018181607F60954D
:100BB000862381830895FC0181816073609586237B
:100BC00081830895FC0186818C7F862B868308951E
:100BD000FC0186818C7F862B86830895FC018681AB
:100BE000837F862B86830895FC018681837F862BF5
:100BF00086830895FC0187818C7F862B87830895E7
:100C0000FC0187818C7F862B87830895FC01878177
:100C1000837F862B87830895FC018781837F862BC2
:100C200087830895FC0187818F7C862B87830895B5
:100C3000FC0187818F73862B87830895FC01808157
:100C4000807F80838CE081870895FC018081807F94
:0C0C500080838CE081870895F894FFCF2A
:080C5C0047200D2038202B2059
:00000001FF
